:020000020000FC
:1000000010C03EC14AC14AC159C14EC14BC14BC1CA
:100010004CC145C145C145C14FC14FC14CC14FC184
:100020004FC1F89400E812E006BD16BD08E00BBB16
:100030000CEB0ABB0CE008BB03EF07BBB0E0A0E68B
:1000400000E00D93B130E9F7A036D9F711E00FE5E4
:100050001EBF0DBF00E000B900E105BF00E000BF1A
:1000600000E003BF00E006BF00E00CBF00E003BDFE
:1000700000E00FBD00E00EBD00E002BD10E000E0BA
:100080001DBD0CBD10E000E01BBD0ABD10E000E08E
:1000900019BD08BD10E000E015BD04BD00E807B9BA
:1000A00007E006B900E103B903E001B900E808B9C7
:1000B000A89504B7017F04BF09E319E301BD11BD91
:1000C00000E70ABF07E008BF07E20BB900E002BB88
:1000D00000E000BD00E40BBF00E009BF00E00CB988
:1000E00000E0E02E90E004E646D109B306FF79C0B7
:1000F00000C0DA9ADB9801E200BF01E003BF09E12A
:100100000CBF00E00FBD05E20EBD00E807B9DCE85A
:10011000C0EA302EA89509B306FF8DC02197D030D4
:1001200009F438C007EC06B904E625D104B105B1DD
:10013000023A80F30FEF0CBFA89509B306FF7BC00E
:100140002197D03009F426C007EC06B904E613D194
:1001500004B105B1013E80F3A89509B306FF6BC059
:100160002197D03009F416C007EC06B904E603D194
:1001700004B105B1013E59F020F00CB70A950CBF4F
:1001800006C00CB70F3F09F003950CBF00C00CB7B9
:10019000053510F7ECBEE9BCE8BC04E6ECD0DB9A10
:1001A00000E003BF00E000BF00E003BF00EC03BFBE
:1001B000DA9800E006B900E007B900E808B90FE0F6
:1001C00000B901B5086101BD077F01BD04EB10EB6B
:1001D00005BF15BFA89509B306FDFCCF0AEFCBD02C
:1001E0002AC0DA9A01E20FBD02E20EBD01E007B9B2
:1001F00007EC06B904E6BFD004B105B100951E2D89
:1002000030E022E3020F131FB12FA02F10E0E9BC52
:1002100018BD05E0B0D01395D1F7A89500E807B94F
:1002200007EC06B904E6A7D004B105B1023B08F417
:1002300002C0119791F7ECBEE9BCE8BC04E69BD084
:10024000DB9A00E003BF00E000BF00E003BF00EC6A
:1002500003BFDA9800E006B900E007B900E808B982
:100260000FE000B901B5086101BD077F01BD04EBD6
:1002700010EB05BF15BF7894889500000000FDCFF6
:1002800004E679D009B306FF01C006C0A89506B3FD
:1002900002FFFCCF04E66FD0C4CE189518951895D0
:1002A00018951895189518951895FFB63A9409F46D
:1002B000C2CFFFBE189518951895189518951895E2
:1002C0001895101718F4021708F400000895201B61
:1002D000310B20F4041B150B08F4000008954F9314
:1002E0005F936F93551B441B61E110F4400F511F46
:1002F00057954795379527956A95B9F75F934F932B
:100300003F932F930F911F912F913F916F915F9189
:100310004F9108954F935F936F934427552760E162
:10032000000F111F441F551F4217530718F0039564
:10033000421B530B6A95A1F75F934F932F913F9107
:100340006F915F914F9108951F93E199FECF10E057
:100350001CBB10E08EBB0DBB753A11F4E29AE19A1A
:100360001F9108951F93E199FECF10E08EBBE09A94
:100370000DB31F9108951F932F932BE119E11A9547
:10038000F1F72A95D9F70A95C1F72F911F91089592
:00000001FF
